:1000000014C02DC02CC02BC02AC029C04FC127C08E
:1000100026C06FC124C023C022C021C020C01FC081
:100020001EC01DC01CC062706D0011241FBECFE534
:10003000D4E0DEBFCDBF10E0A0E6B0E0E4E2F7E040
:1000400002C005900D92A839B107D9F710E0A8E9D0
:10005000B0E001C01D92A33AB107E1F7BEC1D0CF15
:100060008FE081BB82B3806F82BB929889E00000F1
:10007000815087FFFCCF90B39F60929A8FEF81BB36
:10008000892F992708958AE08093A0008CE185BD8F
:1000900080919E00882321F48093980080E91BC002
:1000A00080919E00282F332780919D00E82FFF2705
:1000B000EE0FFF1FE05AFF4F80819181281739070B
:1000C00021F41092980086EB06C0809198008F5F13
:1000D0008093980089ED83BD20919800222321F41C
:1000E000939885B388630FC0939A33272E5F3F4F51
:1000F00081E090E002C0880F991F2A95E2F7982FBF
:10010000909585B3892385BB80919E00482F552704
:1001100080919D00E82FFF27EE0FFF1FE659FF4F4C
:1001200020813181CA010196B90198D280939E0045
:10013000089515BC939A85B3886385BB0895282FCD
:1001400033274427552760E47EE785E090E099D285
:10015000DA01C90101979BBD8ABD1DBC1CBC089575
:1001600080919700882311F0C19A01C0C19860E086
:10017000862FF6D18091A200843648F08091A200AB
:1001800064E660D26AE05ED2892F805D01C080E2C1
:10019000FAD18091A2008A3040F08091A2006AE0FA
:1001A00051D250D2892F805D01C080E2ECD1809184
:1001B000A2006AE047D2892F805DE5D161E080E04E
:1001C000CFD180919D00E82FFF27EE0FFF1FE3574F
:1001D000FF4F80819181E9D1089599278F3B910547
:1001E000A1F0803C910524F48F37910541F00895EA
:1001F0008F3D9105E9F08F3E9105B1F00895809112
:1002000097008095809397000BC080919D0099275F
:10021000019665E070E022D280939D0010929E00CE
:1002200081E08093A10008958091A2008F5F03C0B8
:100230008091A20081508093A2008091A2007FDF74
:10024000EFCF99278F3D9105A9F08F3E910569F574
:100250008091A2002AE0622FF5D18F5F829FC001BA
:1002600011248093A2008091A20069DF81E0809335
:10027000A10008958091A2002AE0622FE3D1992382
:1002800029F48091A200DED1815004C08091A200A7
:10029000622FD8D1829FC00111248093A200809147
:1002A000A2004DDF81E08093A10008951F920F927C
:1002B0000FB60F9211242F933F934F935F936F9339
:1002C0007F938F939F93AF93BF93EF93FF93DBDE67
:1002D000FF91EF91BF91AF919F918F917F916F911E
:1002E0005F914F913F912F910F900FBE0F901F90F4
:1002F00018951F920F920FB60F9211242F933F93D0
:100300004F935F936F937F938F939F93AF93BF931D
:10031000EF93FF9387E882BF8091A000882351F07C
:100320008091A00081508093A0008091A00088233C
:1003300009F4FFDE95DE90919C00891751F48091BD
:100340009A008A3F78F480919A008F5F80939A0098
:1003500009C080919C008093990082DE80939C006C
:1003600010929A0080919A00823059F490919C00EA
:1003700080919900981701F180919C0080939B00D7
:100380001BC080919A008330B8F080919A0029E1D7
:10039000622F58D1992381F490919C00809199000B
:1003A000981751F080919C008F3F31F080919C0014
:1003B00080939F0020939A00FF91EF91BF91AF919E
:1003C0009F918F917F916F915F914F913F912F916D
:1003D0000F900FBE0F901F901895CFE5D4E0DEBFB1
:1003E000CDBF1FEF11BB0CE002BB17BB87EF88BB73
:1003F00014BB8FE385BB87E882BF85E083BF1FBC4A
:100400008DE08EBD84E68093A2008091A20097DEED
:1004100015BE81E189BF1093990080919900809366
:100420009C0010929A0081E08093A100802FDBD085
:10043000A4D060E084E094D086E290E0C3D080E86D
:1004400088B9789480919B00882329F080919B0043
:10045000C4DE10929B0080919F00882329F0809138
:100460009F00EFDE10929F008091A100813051F734
:1004700077DE1092A100E6CFAA9A00C0AA9808954C
:10048000CF93DF93982F662311F0A89A01C0A89804
:10049000A9988C9A8D9A8E9A8F9A979896989598F3
:1004A000949897FD979AC92FDD27C6FD969AC5FDAA
:1004B000959AC4FD949AE0DF9798969895989498A9
:1004C000C3FD979AC2FD969AC1FD959AC0FD949A74
:1004D000D3DF949A959A969A979ADF91CF9108953F
:1004E000882311F0A89A01C0A898A99A8C988D9891
:1004F0008E988F98AA9A00C080E0849980E18599AF
:1005000080628699806487998068AA9800C0AA9AB8
:1005100000C08499816085998260869984608799FA
:100520008860AA989927089580E0DADF8823E4F3A9
:1005300083E090E00197F1F780E0D2DF99270895FA
:100540001F93182FF1DF60E0812F9ADF1F9108952C
:100550001F93182FE9DF61E0812F92DF1F9108952B
:10056000982F662319F4892F805802C0892F805450
:10057000E7DF0895D9DF9927089581E0E1DF089545
:1005800082E0DEDF0895CF93C82FCEDFCA3041F47A
:10059000803410F480E401C080E08058D1DF03C0D3
:1005A00061E08C2F6DDFCF910895CF93DF93EC0145
:1005B0008991882321F0E7DF89918823E1F7DF9192
:1005C000CF910895CF93DF93EC01FC0121968491A4
:1005D000882331F0D8DFFE01219684918823D1F75A
:1005E000DF91CF9108951F93182FA09AA19AA29AF4
:1005F0008C9A8D9A8E9A8F9A80E090E60197F1F707
:10060000959A949A39DF83EF9DE10197F1F734DFF2
:1006100082E690E00197F1F72FDF82E690E0019704
:10062000F1F7949829DF82E690E00197F1F788E2EC
:1006300087DF88E085DFA1DF86E082DF812F80DF32
:100640001F910895991B79E004C0991F961708F02F
:10065000961B881F7A95C9F78095089597FB092EF8
:1006600007260AD077FD04D027D006D000201AF440
:10067000709561957F4F0895F6F7909581959F4FFE
:10068000089597FB092E05260ED057FD04D028D0DB
:100690000AD0001C38F450954095309521953F4F75
:1006A0004F4F5F4F0895F6F790958095709561953F
:1006B0007F4F8F4F9F4F0895AA1BBB1B51E107C06F
:1006C000AA1FBB1FA617B70710F0A61BB70B881FE2
:1006D000991F5A95A9F780959095BC01CD01089571
:1006E000A1E21A2EAA1BBB1BFD010DC0AA1FBB1F36
:1006F000EE1FFF1FA217B307E407F50720F0A21BA8
:10070000B30BE40BF50B661F771F881F991F1A9414
:1007100069F760957095809590959B01AC01BD013E
:04072000CF01089568
:1007240000000000000002000300010002000300BA
:10073400040006006E6F6E6500322F782000332FA0
:10074400782000342F342000362F382000740079AC
:08075400007E0083008800FF15
:00000001FF
